:10000000830100308A0004282030840025300D2030
:100010008301BC2B04068001840A0406031D0A2800
:020020000034AA
:10076C008312A4008312A40BB82B080080308316CC
:10077C0081008B0195019F010130831285000730A8
:10078C009900FE30831685008312D023A000200A26
:10079C00E523CA2B8312851CD02B16308312B6236B
:1007AC00851CD02B0830A200A3011730B6230310F0
:1007BC0085180314A30CA20BDB2B2309080083124E
:1007CC00A3000930A2000508A10021102108850012
:1007DC00000018308312B62323182114231C211077
:1007EC00210885001630B6230314A30CA20BF22BA0
:0207FC000800F3
:02400E00813FF0
:00000001FF
